:100000000C942A000C94EE000C9412010C94450000
:100010000C9445000C9445000C9445000C9445004C
:100020000C9445000C9445000C9445000C9445003C
:100030000C9445000C9445000C9445000C9445002C
:100040000C9445000C9445000C9445000C9445001C
:100050000C94450011241FBECFE5D8E0DEBFCDBF14
:1000600010E0A0E6B0E0ECE6F2E002C005900D92F0
:10007000A037B107D9F710E0A0E7B0E001C01D92AA
:10008000A337B107E1F70C9482000C9400001CBE6A
:1000900013BC8DE683BF85BD089510927200109247
:1000A000710085E085BF80EC8BBF0895882321F423
:1000B000C09A8DE683BF0895C0988DE783BF0895E9
:1000C0000895882311F46CBF0895813009F00895D4
:1000D00063BD08950895CF93DF93EC0118161906B8
:1000E0002CF481E00E9456006C2F06C080E00E9434
:1000F00056008C2F8195682F80E00E946100DF916F
:10010000CF910895CFE5D8E0DEBFCDBF1ABA89E020
:1001100087BB14BA80E881BB0E9447000E944D0053
:1001200078948091710090917200AA2797FDA09514
:10013000BA2F8F3F9105A105B10529F024F08FEF6B
:1001400090E0A0E0B0E081302FEF92072FEFA20700
:100150002FEFB20724F481E09FEFAFEFBFEF0E94D3
:100160006B00DFCFCF93DF93EC011816190654F420
:1001700060E0862F0E94610081E00E9456006C2F93
:1001800081E00BC060E081E00E94610080E00E949D
:1001900056008C2F8195682F80E00E946100DF91CE
:1001A000CF91089540B34C7080917000482BE0E6E9
:1001B000F0E0E40FF11D8081992787FD9095209153
:1001C000710030917200820F931F909372008093A0
:1001D0007100469546954093700008951F920F92C6
:1001E0000FB60F9211242F933F934F935F936F930A
:1001F0007F938F939F93AF93BF93EF93FF930E944F
:10020000D200FF91EF91BF91AF919F918F917F911C
:100210006F915F914F913F912F910F900FBE0F9073
:100220001F9018951F920F920FB60F9211242F93C3
:100230003F934F935F936F937F938F939F93AF936E
:10024000BF93EF93FF930E94D200FF91EF91BF9174
:10025000AF919F918F917F916F915F914F913F915E
:0C0260002F910F900FBE0F901F9018956B
:10026C000001FF00FF000001010000FF00FF010082
:00000001FF
